:100000003F28A301A200FF30A207031CA307031C83
:100010003A280330A100E6300F200328A101FC3E5E
:10002000A000A109031C1A28FF300000A007031834
:100030001528A0076400A10F14280800A501A40139
:100040001030A600210DA40DA50D2208A40223083E
:10005000031C230FA502031834282208A407230831
:100060000318230FA5070310A00DA10DA60B22282E
:1000700020083A28831303138312640008008316B0
:1000800007309C008601F030850010309B008030E6
:100090009F008312E5309F001F1505308A010E2056
:1000A00064008A111F194D281E08B90083161E0806
:1000B0008312B800BD01BD0A64003D08643C8A118A
:1000C00003194C283808BA003908BB003A08A000C8
:1000D0003B08A100E830A2000330A3008A011E20E3
:1000E000BC003A08A0003B08A100E830A2000330A1
:1000F000A3008A011E202408BA002508BB008A112B
:10010000E1203C0886000830850001308A0101208A
:1001100085013A08A0003B08A1006430A200A301B9
:100120008A011E20BC003A08A0003B08A1006430F0
:10013000A200A3018A011E202408BA002508BB00E2
:100140008A11E1203C0886000430850001308A01D4
:10015000012085013A08A0003B08A1000A30A20056
:10016000A3018A011E20BC003A08A0003B08A100A0
:100170000A30A200A3018A011E202408BA00250823
:10018000BB008A11E1203C08860001308500013067
:100190008A01012085013A08BC008A11E1203C084F
:1001A00086000230850001308A0101208501FD3082
:1001B00086000130850001308A01012085018A0115
:1001C0005B283C08093C8A11031CF9288A11EB20A2
:1001D000BC008A11F92800308A003C0882072234CA
:1001E0007B3416341A344B348A34C2343B340234F0
:0A01F0000B34080063008A01FA28AE
:02400E00623F0F
:00000001FF
